:100000000C9434000C9446000C9448000C94460068
:100010000C9446000C9446000C9446000C94460048
:100020000C9446000C9446000C9446000C94460038
:100030000C9446000C9446000C9446000C94460028
:100040000C9446000C9446000C9446000C94460018
:100050000C9446000C9446000C9446000C94460008
:100060000C9446000C94460011241FBECFEFD8E03C
:10007000DEBFCDBF21E0A0E0B1E001C01D92A13004
:10008000B207E1F70E9457000C9473000C94000033
:100090001F920F920FB60F9211248F9381E08093DD
:1000A00000018F910F900FBE0F901F9018958091B7
:1000B00069008F60809369008DB383608DBB8FB7BB
:1000C00080688FBF8FEF87B921E092E080910001B7
:1000D000882329F088B1822788B91092000188B15D
:0A00E000892788B9F3CFF894FFCF09
:00000001FF
